:020000040000FA
:06000000FBEF18F01200F6
:020006001200E6
:0600080093EF11F012005D
:02000E00C2909E
:040010009D9C1200A1
:04001400B46A1200B8
:06001800EEEF11F01200F2
:02001E000400DC
:1000200061320000FF0700000100000060320000A4
:10003000FF060000010000005F320000FF05000025
:10004000010000005E320000FF040000010000001B
:10005000D9CFE6FFE1CFD9FFFD0EDBCFA1F0FE0E39
:10006000DBCFA2F0A1C0E9FFA2C0EAFF000EEE6E56
:100070000B0EED6EA1C0E9FFA2C0EAFF020EEB6A13
:10008000030EEB6AA1C0E9FFA2C0EAFF060EE92653
:10009000000EEA22EF6AA1C0E9FFA2C0EAFF040E47
:1000A000E926000EEA22050EEF6EA1C0E9FFA2C00C
:1000B000EAFF080EE926000EEA22EF6AA1C0E9FF76
:1000C000A2C0EAFF050EE926000EEA22EF6AA1C0EF
:1000D000E9FFA2C0EAFF020EEB6A030EEB6AA1C0C1
:1000E000E9FFA2C0EAFF090EE926000EEA22EF6A44
:1000F000A1C0E9FFA2C0EAFF0B0EE926000EEA222A
:10010000EF6AA1C0E9FFA2C0EAFF0C0EE926000ECB
:10011000EA22EF6AA1C0E9FFA2C0EAFF0F0EE926BA
:10012000000EEA22EF6AA1C0E9FFA2C0EAFF0D0EAD
:10013000E926000EEA22EF6AA1C0E9FFA2C0EAFFA9
:100140000E0EE926000EEA22220EEF6EE552E7CFF0
:10015000D9FF1200A1C0E9FFA2C0EAFF0F0EE926F5
:10016000000EEA22110EEF6E94869488C76AC66A62
:10017000C56AF00EC6140809C66E630EC86EC78E37
:10018000C68A1200D9CFE6FFE1CFD9FF020EE126E1
:10019000FD0EDB506FE0DE6ADD6ADECF10F0DDCFF2
:1001A00011F0FD0EDB50000111AE02D0D89003D04B
:1001B000105C000E115826E2FB0EDBCF12F0FC0E95
:1001C000DBCF13F0DE501224E96EDD501320EA6E0F
:1001D000EF50E66EDECF10F0DDCF11F0A1C0E9FFE9
:1001E000A2C0EAFF1050EE24E76E1150EE20EA6E36
:1001F000E7CFE9FFE552E750EF6EDF2A010ECDE3CE
:10020000DB2ACBD7FD0EDB50E66EA1C0E9FFA2C012
:10021000EAFF020EE926000EEA22E552E750EE6EF2
:10022000ED6AA1C0E9FFA2C0EAFF0D0EE926000EAB
:10023000EA22FE0EDBCFEFFFA1C0E9FFA2C0EAFF7A
:10024000050EE926000EEA22EF6AA1C0E9FFA2C06E
:10025000EAFF040EE926000EEA22090EEF6EA1C0A5
:10026000E9FFA2C0EAFF0E0EE926000EEA22200EE8
:10027000EF6EC580020EE15C02E2E16AE552E16EDA
:10028000E552E7CFD9FF1200D9CFE6FFE1CFD9FF82
:10029000FD0EDB5038E0FD0EDB50E66EA1C0E9FF3D
:1002A000A2C0EAFF020EE926000EEA22E552E7505C
:1002B000EE6EED6AA1C0E9FFA2C0EAFF0D0EE926CD
:1002C000000EEA22FE0EDBCFEFFFA1C0E9FFA2C0C5
:1002D000EAFF050EE926000EEA22EF6AA1C0E9FF57
:1002E000A2C0EAFF040EE926000EEA22090EEF6E14
:1002F000A1C0E9FFA2C0EAFF0E0EE926000EEA2225
:10030000210EEF6EC580E552E7CFD9FF1200D9CF9D
:10031000E6FFE1CFD9FFA1C0E9FFA2C0EAFF0F0EBF
:10032000E926000EEA22100EEF6E94869488FE0EE7
:10033000DB50E824C86EC76AC66AC56AF00EC614E8
:100340000E09C66EC78EC580C68AE552E7CFD9FFB3
:100350001200A1C0E9FFA2C0EAFF0F0EEB50110886
:1003600002E1BDEF01F0A1C0E9FFA2C0EAFF0F0E5C
:10037000EB50100801E1E4D91200A1C0E9FFA2C0CE
:10038000EAFF0E0EEB50200801E09DD0A1C0E9FF6E
:10039000A2C0EAFF040EEB500B0A19E0020A04E0C7
:1003A0000C0A01E18FD01200A1C0E9FFA2C0EAFF50
:1003B000040EE926000EEA220B0EEF6EA1C0E9FF43
:1003C000A2C0EAFF0D0EEB50E824C96E1200C5BCB6
:1003D00058D0A1C0E9FFA2C0EAFF050EEB50106E95
:1003E000116A020EE926000EEA22EECF12F0EFCFDC
:1003F00013F011501318E8AE02D0133404D0125089
:10040000105C135011581BE2A1C0E9FFA2C0EAFF23
:10041000050EEB50116AE850EE24E76E1150EE2005
:10042000EA6EE7CFE9FFEF50C96EA1C0E9FFA2C0B5
:10043000EAFF050EE926000EEA22EF2A1200A1C00B
:10044000E9FFA2C0EAFF040EE926000EEA22050E2B
:10045000EF6EC584A1C0E9FFA2C0EAFF0E0EE92637
:10046000000EEA22220EEF6E000EE66EE66A2B0EFA
:10047000E66EE66A80EC09F0E552E552E552E55297
:100480001200A1C0E9FFA2C0EAFF040EE926000E97
:10049000EA22050EEF6EC584A1C0E9FFA2C0EAFF03
:1004A0000E0EE926000EEA22220EEF6E000EE66E18
:1004B000E66A2C0EE66EE66A80EC09F0E552E5523B
:1004C000E552E5521200A1C0E9FFA2C0EAFF0E0EFC
:1004D000EB50210801E0D7D0A1C0E9FFA2C0EAFF9C
:1004E000040EEB500D0A01E19FD0010A01E190D00A
:1004F0000B0A40E00C0A1AE0020A04E00C0A01E1CF
:10050000C2D01200A1C0E9FFA2C0EAFF040EE92692
:10051000000EEA220B0EEF6EA1C0E9FFA2C0EAFFB7
:100520000D0EEB50E8240109C96E1200C5AC70D065
:10053000A1C0E9FFA2C0EAFF040EE926000EEA22EC
:10054000050EEF6EC584A1C0E9FFA2C0EAFF0E0E42
:10055000E926000EEA22220EEF6E000EE66EE66A33
:100560002E0EE66EE66A80EC09F0E552E552E552A1
:10057000E5521200A1C0E9FFA2C0EAFF050EEB5050
:10058000116AE850EE24E76E1150EE20EA6EE7CFD4
:10059000E9FFC9CFEFFFA1C0E9FFA2C0EAFF050E46
:1005A000E926000EEA22EF2AA1C0E9FFA2C0EAFF75
:1005B000050EEB50106E116A020EE926000EEA22BB
:1005C000EECF12F0EFCF13F011501318E8AE02D0B7
:1005D000133404D01250105C135011580CE2A1C017
:1005E000E9FFA2C0EAFF040EE926000EEA220C0E83
:1005F000EF6EC59A0BD0A1C0E9FFA2C0EAFF040EBE
:10060000E926000EEA220D0EEF6EC58AC58812009B
:10061000A1C0E9FFA2C0EAFF040EE926000EEA220B
:10062000070EEF6EC5861200A1C0E9FFA2C0EAFF67
:10063000040EE926000EEA22050EEF6EC584A1C065
:10064000E9FFA2C0EAFF0E0EE926000EEA22220E02
:10065000EF6EA1C0E9FFA2C0EAFFEECFE6FFEFCF49
:10066000E6FF2D0EE66EA1C0E9FFA2C0EAFF020E72
:10067000E926000EEA22EF50E66E80EC09F0E55222
:10068000E552E552E5521200D9CFE6FFE1CFD9FF9E
:10069000A1C0E9FFA2C0EAFF060EE926000EEA2289
:1006A000010EEF6EA1C0E9FFA2C0EAFF020EEB6AE5
:1006B000030EEB6AFE0EDB5035E0C7AA1DD0A1C0C9
:1006C000E9FFA2C0EAFF040EE926000EEA22050EA9
:1006D000EF6EA1C0E9FFA2C0EAFF080EE926000EF6
:1006E000EA22EF2AA1C0E9FFA2C0EAFF070EE9262D
:1006F000000EEA22050E1FD0C7A40AD0A1C0E9FF50
:10070000A2C0EAFF040EE926000EEA22080E13D06A
:10071000A1C0E9FFA2C0EAFF040EE926000EEA220A
:10072000070E09D0A1C0E9FFA2C0EAFF040EE92626
:10073000000EEA22060EEF6EE552E7CFD9FF120057
:10074000D9CFE6FFE1CFD9FF090EE126010EDB6A22
:10075000020EDB6A030EDB6A040EDB6A080EDB6A3C
:10076000C6AC23D0C69CA1C0E9FFA2C0EAFF040E1C
:10077000E926000EEA22050EEF6E010EF36E040E5E
:10078000F3CFDBFFA1C0E9FFA2C0EAFF080EE92614
:10079000000EEA22EF2AA1C0E9FFA2C0EAFF070E7D
:1007A000E926000EEA22040EEF6EC7A005D0C9505C
:1007B000DF6EDE52010EDD6E040EDB5001E024D24E
:1007C000A1C0E9FFA2C0EAFF040EEB50070A01E155
:1007D00060D10F0A6CE00E0A14E0030A01E014D2A3
:1007E000C7A612D2010EDBCFE6FF4EDFE552A1C055
:1007F000E9FFA2C0EAFF040EEB50080801E004D2B2
:1008000037D0C7A810D0A1C0E9FFA2C0EAFF060EEA
:10081000E926000EEA22EF2A010EDB5001E1EAD1BF
:10082000C7AA89D1D4D1010EDB5001E1EDD1A1C01D
:10083000E9FFA2C0EAFF060EE926000EEA22EF2A2F
:10084000C7BA18D0C7B40AD0A1C0E9FFA2C0EAFF56
:10085000040EE926000EEA22070ED5D1A1C0E9FF59
:10086000A2C0EAFF040EE926000EEA22080EEF6E8F
:10087000030EABD1A1C0E9FFA2C0EAFF080EE92632
:10088000000EEA22EF2AA1C0E9FFA2C0EAFF040E8F
:10089000E926000EEA22050EEF6EA1C0E9FFA2C014
:1008A000EAFF070EE926000EEA22060EACD1A1C02F
:1008B000E9FFA2C0EAFF0B0EEB50000901E080D077
:1008C00047EC0AF0E76E080EE7CFDBFFDB502A08A3
:1008D00003E1080EDB501BE1C968A1C0E9FFA2C01B
:1008E000EAFF050EE926000EEA22010EEF6EA1C016
:1008F000E9FFA2C0EAFF0B0EE926000EEA22010E74
:10090000EF6EA1C0E9FFA2C0EAFF0C0E53D0A1C058
:10091000E9FFA2C0EAFFEECFE6FFEFCFE6FFA1C0FE
:10092000E9FFA2C0EAFF0A0EEB50E66EE66AE6684F
:1009300027EC0AF0126E050EE15E1250106E116A7D
:1009400010BE1168A1C0E9FFA2C0EAFF020E10C0EC
:10095000EBFF030E11C0EBFFA1C0E9FFA2C0EAFF4D
:10096000020EE926000EEA22EECF10F0EFCF11F0D2
:10097000113401E349D110500008000E115401E375
:1009800043D1A1C0E9FFA2C0EAFFEE50EFCFEAFFDA
:10099000E96EEF50C96EA1C0E9FFA2C0EAFF050EE3
:1009A000E926000EEA22010EEF6EA1C0E9FFA2C007
:1009B000EAFF0B0EE926000EEA22010EEF6E5AD076
:1009C000A1C0E9FFA2C0EAFF0C0EEB5000091CE039
:1009D000A1C0E9FFA2C0EAFF050EEB50106E090EA0
:1009E000EB50105C02E2C9683BD0A1C0E9FFA2C095
:1009F000EAFF0B0EE926000EEA22EF6AA1C0E9FF2A
:100A0000A2C0EAFF0C0E40D0A1C0E9FFA2C0EAFFDD
:100A1000050EEB50106E116A020EE926000EEA2256
:100A2000EECF12F0EFCF13F011501318E8AE02D052
:100A3000133404D01250105C1350115820E2A1C09E
:100A4000E9FFA2C0EAFF050EEB50116AE850EE2460
:100A5000E76E1150EE20EA6EE7CFE9FFEF50C96E66
:100A6000A1C0E9FFA2C0EAFF050EE926000EEA22B6
:100A7000EF2A010EF36E020EF3CFDBFFC5D0A1C04B
:100A8000E9FFA2C0EAFF0B0EE926000EEA22EF6A98
:100A9000B1D0C7A856D0A1C0E9FFA2C0EAFF060E98
:100AA000E926000EEA22EF2A010EDB5044E0C7AA35
:100AB00025D0A1C0E9FFA2C0EAFFEECF10F0EFCF32
:100AC00011F0A1C0E9FFA2C0EAFF020EE926000E64
:100AD000EA221050EE24E76E1150EE20EA6EE7CFC6
:100AE000E9FFDFCFEFFFA1C0E9FFA2C0EAFF020EDE
:100AF000E926000EEA22EE2AEF221DD0A1C0E9FF6E
:100B0000A2C0EAFF080EE926000EEA22EF2AA1C0E1
:100B1000E9FFA2C0EAFF070EE926000EEA22060E50
:100B2000EF6EA1C0E9FFA2C0EAFF040EE926000EA5
:100B3000EA22050E5ED0010EF36E030EF3CFDBFF4B
:100B400059D0010EDB5060E0A1C0E9FFA2C0EAFF6E
:100B5000060EE926000EEA22EF2AC7AA25D0A1C078
:100B6000E9FFA2C0EAFFEECF10F0EFCF11F0A1C075
:100B7000E9FFA2C0EAFF020EE926000EEA221050A9
:100B8000EE24E76E1150EE20EA6EE7CFE9FFDFCFEB
:100B9000EFFFA1C0E9FFA2C0EAFF020EE926000EA6
:100BA000EA22EE2AEF2230D0C7A411D0A1C0E9FF7B
:100BB000A2C0EAFF040EE926000EEA22080EEF6E3C
:100BC000010EF36E030EF3CFDBFFC96E1DD0A1C083
:100BD000E9FFA2C0EAFF080EE926000EEA22EF2A8A
:100BE000A1C0E9FFA2C0EAFF070EE926000EEA2233
:100BF000060EEF6EA1C0E9FFA2C0EAFF040EE926CF
:100C0000000EEA22050EEF6E010EDB5003E1020E2C
:100C1000DB5002E0C6A8C688A1C0E9FFA2C0EAFF77
:100C2000020EE926000EEA22EECF10F0EFCF11F00F
:100C3000113425E21050FD08000E115420E2030E7D
:100C4000DB501DE1A1C0E9FFA2C0EAFF040EE926C6
:100C5000000EEA22050EEF6EA1C0E9FFA2C0EAFF76
:100C6000080EE926000EEA22EF2AA1C0E9FFA2C081
:100C7000EAFF070EE926000EEA22070EEF6E030ECA
:100C8000DB506DE0A1C0E9FFA2C0EAFF020EE92639
:100C9000000EEA22EECF10F0EFCF11F01006115A3D
:100CA000A1C0E9FFA2C0EAFF1050EE24E76E115088
:100CB000EE20EA6EE7CFE9FFEF50E66EA1C0E9FF54
:100CC000A2C0EAFF090EE926000EEA22E552E7502B
:100CD000EF6EA1C0E9FFA2C0EAFF060EEB50E66E80
:100CE000EECF10F0EFCF11F0A1C0E9FFA2C0EAFFF4
:100CF000020EE926000EEA221050EE24E76E115093
:100D0000EE20EA6EE7CFE9FFE552E750EF6EA1C0B3
:100D1000E9FFA2C0EAFFEECFE6FFEFCFE6FF290E24
:100D2000E66EA1C0E9FFA2C0EAFF020EE926000EAE
:100D3000EA22EECF10F0EFCF11F0010E1024E66E94
:100D400080EC09F0E552E552E552E552A1C0E9FF19
:100D5000A2C0EAFF020EEB6A030EEB6A38D0A1C014
:100D6000E9FFA2C0EAFF080EEB50106E010E105C06
:100D70002EE3A1C0E9FFA2C0EAFF080EEB50E76E28
:100D8000050EE7CFDBFF070EEB50E76E060EE7CF51
:100D9000DBFFEB50E76E070EE7CFDBFFD950050F07
:100DA000E66E000EDA20E66E280EE66E030EE66EA4
:100DB00080EC09F0E552E552E552E552A1C0E9FFA9
:100DC000A2C0EAFF080EE926000EEA22EF6A090E29
:100DD000E15C02E2E16AE552E16EE552E7CFD9FF5C
:100DE0001200A1C0E9FFA2C0EAFF0E0EEB502208DC
:060DF00001E1000C010C02
:0A0DF600D9CFE6FFE1CFD9FFE652A6
:100E0000FD0EDBCFE9FFFE0EDBCFEAFF0A0EE9267F
:100E1000000EEA22EF6AFD0EDBCFE9FFFE0EDBCF0C
:100E2000EAFF0B0EE926000EEA22EF6ADF6A020EE5
:100E3000DF5C11E2FD0EDBCFE9FFFE0EDBCFEAFF48
:100E4000DF50050DE950F324E96EEA50F420EA6E14
:100E5000EF6ADF2AECD7E552E552E7CFD9FF12005F
:100E60000001906B000E636F090E646F000E686FD7
:100E7000080E696F000E6F6F070E706F000E746FB3
:100E8000060E756F000E7B6F050E7C6F000E806F77
:100E9000040E816F000E876F030E886F000E8C6F3B
:100EA000020E8D6F600EE66E000EE66EA4DFE55258
:100EB000E5526C0EE66E000EE66E9DDFE552E552E1
:100EC000780EE66E000EE66E96DFE552E552840E71
:100ED000E66E000EE66E8FDFE552E5521200D9CFC6
:100EE000E6FFE1CFD9FF050EE126FC0EDB50E66EF2
:100EF000D950030FE96EDACFEAFFE552E750EE6E04
:100F0000ED6AFD0EDBCFE9FFFE0EDBCFEAFF0A0E36
:100F1000E926000EEA22EFCFDFFFFD0EDBCFE9FF6F
:100F2000FE0EDBCFEAFFE9CF12F0EACF13F0DF507D
:100F3000050DE950F324106EEA50F420116E010EF5
:100F400010C0DBFF020E11C0DBFF010EDBCFE9FF9B
:100F5000020EDBCFEAFFEF5002E0FF0E58D0010E89
:100F6000DBCFE9FF020EDBCFEAFFEE52FC0EDBCF58
:100F7000EFFF010EDBCFE9FF020EDBCFEAFFE92630
:100F8000000EEA22FB0EDBCFEFFF030EDBCFE6FF06
:100F9000040EDBCFE6FFF90EDBCFE6FFFA0EDBCF68
:100FA000E6FF010EDBCFE9FF020EDBCFEAFF030E07
:100FB000E926000EEA22EECFE6FFEFCFE6FF7AEC5D
:100FC00017F0106E060EE15E1050FD0EDBCFE9FF4C
:100FD000FE0EDBCFEAFF0A0EE926000EEA22EF281A
:100FE000010BE66EFD0EDBCFE9FFFE0EDBCFEAFF65
:100FF0000A0EE926000EEA22E552E750EF6E010ED6
:10100000DBCFE9FF020EDBCFEAFF010EEF6E106EC1
:10101000050EE15C02E2E16AE552E16E1050E55234
:10102000E7CFD9FF1200D9CFE6FFE1CFD9FF050EF8
:10103000E126FD0EDBCFE9FFFE0EDBCFEAFF0B0E54
:10104000E926000EEA22EFCFDFFFFD0EDBCFE9FF3E
:10105000FE0EDBCFEAFFE9CF12F0EACF13F0DF504C
:10106000050DE950F324106EEA50F420116E010EC4
:1010700010C0DBFF020E11C0DBFF010EDBCFE9FF6A
:10108000020EDBCFEAFFEF0401E07AD0010EDBCFE6
:10109000E9FF020EDBCFEAFFEE52EFCF10F0FC0EBD
:1010A000DB50D880105402E2FD0E6BD0010EDBCF76
:1010B000E9FF020EDBCFEAFFEE52EF50E66ED950A9
:1010C000030FE96EDACFEAFFE552E750EE6EED6A04
:1010D000030EDBCFE6FF040EDBCFE6FF010EDBCF16
:1010E000E9FF020EDBCFEAFF030EE926000EEA223B
:1010F000EECFE6FFEFCFE6FFF80EDBCFE6FFF90E0F
:10110000DBCFE6FF7AEC17F0106E060EE15E1050B2
:10111000FD0EDBCFE9FFFE0EDBCFEAFF0B0EE9266B
:10112000000EEA22EF28010BE66EFD0EDBCFE9FF91
:10113000FE0EDBCFEAFF0B0EE926000EEA22E55297
:10114000E750EF6E010EDBCFE9FF020EDBCFEAFFC7
:10115000E926000EEA22EF50E66EFA0EDBCFE9FF39
:10116000FB0EDBCFEAFFE552E750EF6E010EDBCF5F
:10117000E9FF020EDBCFEAFFEF6A030EDB5001D07E
:10118000FC0E106E050EE15C02E2E16AE552E16ED2
:101190001050E552E7CFD9FF1200D9CFE6FFE1CFDB
:1011A000D9FF030EE126FD0EDBCFE9FFFE0EDBCFFC
:1011B000EAFF0B0EE926000EEA22EFCFDFFFFD0E5D
:1011C000DBCFE9FFFE0EDBCFEAFFDF50050DE95074
:1011D000F324106EEA50F420116E010E10C0DBFFF4
:1011E000020E11C0DBFF010EDBCFE9FF020EDBCFE9
:1011F000EAFFEF040BE1010EDBCFE9FF020EDBCFCC
:10120000EAFFE926000EEA22EF5001D0000E106E30
:10121000030EE15C02E2E16AE552E16E1050E55234
:10122000E7CFD9FF1200D9CFE6FFE1CFD9FFFD0EFE
:10123000DBCFE9FFFE0EDBCFEAFFE9CF10F0EACF0C
:1012400011F0FD0EDBCFE9FFFE0EDBCFEAFF0B0E48
:10125000E926000EEA22EF50050D1050F324E96E46
:101260001150F420EA6EEF50E552E7CFD9FF12009B
:10127000D38E03001200D9CFE6FFE1CFD9FFFB0EDA
:10128000DBCFE6FFFC0EDBCFE6FFFD0EDBCFE6FF9C
:10129000FE0EDBCFE6FF600EE66E000EE66E1FDE92
:1012A000106E060EE15E1050E552E7CFD9FF120036
:1012B000D9CFE6FFE1CFD9FFFA0EDBCFE6FFFB0E79
:1012C000DBCFE6FFFC0EDBCFE6FFFD0EDBCFE6FF5C
:1012D000FE0EDBCFE6FF600EE66E000EE66EA3DECE
:1012E000106E070EE15E1050E552E7CFD9FF1200F5
:1012F000600EE66E000EE66E50DFE552E55212001B
:10130000D9CFE6FFE1CFD9FFFB0EDBCFE6FFFC0E26
:10131000DBCFE6FFFD0EDBCFE6FFFE0EDBCFE6FF09
:101320006C0EE66E000EE66EDADD106E060EE15E05
:101330001050E552E7CFD9FF1200D9CFE6FFE1CF39
:10134000D9FFFA0EDBCFE6FFFB0EDBCFE6FFFC0E8C
:10135000DBCFE6FFFD0EDBCFE6FFFE0EDBCFE6FFC9
:101360006C0EE66E000EE66E5EDE106E070EE15E3F
:101370001050E552E7CFD9FF12006C0EE66E000E5A
:10138000E66E0BDFE552E5521200D9CFE6FFE1CF62
:10139000D9FFFB0EDBCFE6FFFC0EDBCFE6FFFD0E39
:1013A000DBCFE6FFFE0EDBCFE6FF780EE66E000E2B
:1013B000E66E95DD106E060EE15E1050E552E7CF49
:1013C000D9FF1200D9CFE6FFE1CFD9FFFA0EDBCF6C
:1013D000E6FFFB0EDBCFE6FFFC0EDBCFE6FFFD0EEC
:1013E000DBCFE6FFFE0EDBCFE6FF780EE66E000EEB
:1013F000E66E19DE106E070EE15E1050E552E7CF83
:10140000D9FF1200780EE66E000EE66EC6DEE552DB
:10141000E5521200D9CFE6FFE1CFD9FFFB0EDBCFBB
:10142000E6FFFC0EDBCFE6FFFD0EDBCFE6FFFE0E98
:10143000DBCFE6FF840EE66E000EE66E50DD106E2A
:10144000060EE15E1050E552E7CFD9FF1200D9CF6A
:10145000E6FFE1CFD9FFFA0EDBCFE6FFFB0EDBCFD5
:10146000E6FFFC0EDBCFE6FFFD0EDBCFE6FFFE0E58
:10147000DBCFE6FF840EE66E000EE66ED4DD106E66
:10148000070EE15E1050E552E7CFD9FF1200840E3F
:10149000E66E000EE66E81DEE552E55212000001B6
:1014A000905101E1120075EC11F0F3CF10F0F4CF80
:1014B00011F0F350F41001E0120059EC11F0F3CFE9
:1014C00010F0F4CF11F0F350F41001E112006C0EA3
:1014D000E66E000EE66EA7DEE552E552000901E079
:1014E0001200600EE66E000EE66E9DDEE552E552DD
:1014F000000901E0120038EF09F081EC11F0F3CFA0
:1015000010F0F4CF11F0F350F41001E112000001DB
:10151000010E906F6C0EE66E000EE66E84DEE552F4
:10152000E552000909E1600EE66E000EE66E7BDE14
:10153000E552E552000903E00001906B12000A0E2B
:0A154000E66EDBEC18F0E552E5D78B
:06154A00D9CFE6FFE1CF5E
:10155000D9FF3B0EE126230EDB6A240EDB6A250E43
:10156000DB6A260EDB6A9B8C8F0ED3147009D36E58
:10157000FC0ED3140009D36E0F0148691F0E496F8A
:1015800062EC16F0D9CFE6FFDACFE6FF8BEC0DF078
:10159000E552E552D950090FE66E000EDA20E66EEC
:1015A00028EC00F0E552E552D950190FE66E000E16
:1015B000DA20E66EA0EC0FF0E552E55230EC07F0D1
:1015C000A6EC14F062EC12F024EC14F02AEC16F005
:1015D00055EC11F04AEC11F0AAEC00F062EC13F0BB
:1015E000E66872EC18F0E55253EC16F07DEC0AF068
:1015F000000EE66E0A0EE66ED950220FE66E000E61
:10160000DA20E66EE6689DEC09F0106E050EE15EEC
:101610001050E76E210EE7CFDBFFDBCF10F0103468
:1016200021E3210EDB50FC08000EE66E0A0EE66E8A
:10163000D950220FE66E000EDA20E66EE66858EC0E
:1016400009F0106E050EE15E1050E76E210EE7CF37
:10165000DBFFDBCF10F0103401E281D1210EDB5033
:10166000FC08C4D7220EDB50440A01E148D1070A26
:1016700001E13BD1010A01E135D1030A01E12FD19A
:10168000010A01E129D17F0A01E123D1010A01E127
:101690001DD1030A01E1D7D0010A01E1BBD0120A32
:1016A000A5E0030A01E182D0010AA0E0070A9EE05A
:1016B000020A13E0010A02E0360A98D7230EDB6A19
:1016C000210EDB50F36E230EDBCFF4FFF350F45CFE
:1016D00001E38CD7230EDB2AF3D7230EDB6A210E1E
:1016E000DB04F36E230EDBCFF4FFF350F45C03E274
:1016F000230EDB2AF4D70A010051090A01E176D74B
:10170000010A01E173D70F0A01E170D7010A01E173
:101710006DD7020A19E0060A01E068D7010EF36EE0
:10172000210EF3CFDBFFD9501D0FE96EDACFEAFFB0
:10173000FF0ED880EE54000EED5402E2006929D06D
:101740001D0EDBCF00FA25D0D9501D0FE96EDACF80
:10175000EAFFFF0ED880EE54000EED5408E2210E91
:10176000DB68000EE66E0A0EE66EE6680DD01D0E12
:10177000DB50E76E210EE7CFDBFF000EE66E0A0EB0
:10178000E66E1D0EDBCFE6FFBEEC10F0E552E55233
:10179000E552000EE66E0A0EE66E2A0EE66E210E89
:1017A000DBCFE6FF0AEC0AF0E55231D0230EDB6A0C
:1017B000210EDB50F36E230EDBCFF4FFF350F45C0D
:1017C00003E2230EDB2AF4D735EC11F0F3CF10F04F
:1017D000F4CF11F0070EF35C000EF45801E206D7C7
:1017E000250EDB0402E10A0E06D0250EDB500208AE
:1017F00001E0FCD60B0EE66ED0EC0FF0E552000EC9
:10180000E66E0A0EE66E060EE66E36EC10F0E55257
:10181000E5525AD0D950270FE96EDACFEAFF000E11
:10182000EE6E0A0EED6E230EDB6A210EDB50FB0F0F
:10183000F36E230EDBCFF4FFF350F45C01E3D6D656
:10184000230EDB2AF2D7D950290FE96EDACFEAFF4F
:10185000000EEE6E0A0EED6E230EDB6A210EDB50DB
:10186000F40FF36E230EDBCFF4FFF350F45C03E2CE
:10187000230EDB2AF3D7290EDBCFE9FF2A0EDBCFBD
:10188000EAFF0C0EE926000EEA22E9CF10F0EACFBB
:1018900011F0E9CFE6FFEACFE6FF210EDB50F40FAF
:1018A000E66E36EC10F0E552E552E552290EDBCF3C
:1018B000E9FF2A0EDBCFEAFF0C0EE926000EEA2232
:1018C000EF50E66EADEC12F0E55290D6D9502B0FEA
:1018D0000ED0D9502D0F0BD0D9502F0F08D0D95082
:1018E000310F05D0D950330F02D0D950350FE96EE2
:1018F000DACFEAFF000EEE6E0A0EED6E77D6D95003
:10190000370FE96EDACFEAFF000EEE6E0A0EED6ECB
:10191000370EDBCFE9FF380EDBCFEAFFEE52EF5098
:10192000110A01E163D6160A01E160D6010A01E15C
:101930005DD6050A01E15AD6010A09E0030A01E170
:1019400055D6010A01E052D6260EDB6A4FD6010EAB
:10195000F36E260EF3CFDBFF60EC16F047D6220EB7
:10196000DB500B0A31E0010A2CE05A0A01E13ED6B5
:101970001D0A24E0010A1FE0070A20E0010A1BE01B
:10198000030A16E0010A0FE00F0A08E0010A01E06D
:10199000B3D0D5EC18F0F7EC14F028D600EC15F025
:1019A000250EDB6A0BD0D5EC18F017EC15F01ED61F
:1019B0001EEC15F003D0D5EC18F018D6D4EC14F0CA
:1019C00015D6CAEC18F012D6D950390FE96EDACF15
:1019D000EAFF000EEE6E0A0EED6E390EDBCFE9FF68
:1019E0003A0EDBCFEAFF100EEF6E390EDBCFE9FFC8
:1019F0003A0EDBCFEAFFEE52EF6A390EDBCFE9FF9A
:101A00003A0EDBCFEAFF020EE926000EEA22EE6A6A
:101A1000EE6AEE6AEE6A390EDBCFE9FF3A0EDBCFF3
:101A2000EAFF020EE926000EEA22040EE926000E65
:101A3000EA22EE6AEE6AEE6AEE6A390EDBCFE9FF61
:101A40003A0EDBCFEAFF0A0EE926000EEA22EE6A22
:101A5000ED6A390EDBCFE9FF3A0EDBCFEAFF0C0E61
:101A6000E926000EEA22EF6A390EDBCFE9FF3A0ED3
:101A7000DBCFEAFF0D0EE926000EEA22010EEF6E23
:101A8000390EDBCFE9FF3A0EDBCFEAFF0E0EE92677
:101A9000000EEA22240EDBCFEFFFDBCFE6FFADEC3A
:101AA00012F0E552240EDB2ADB50640802E1240E1A
:101AB000DB6A0F0EF36E210EF3CFDBFFDBCFE6FF09
:101AC000000EE66E0A0EE66E0EEC0FF0E552E552E1
:101AD000E552250EDB50020807E0250EDB0404E189
:101AE000DDEC13F0020E03D0B3EC13F0010EF36E35
:101AF000250EF3CFDBFF7AD5230EDB6A210EDB50F8
:101B0000F36E230EDBCFF4FFF350F45C01E36ED5EC
:061B1000230EDB2AF3D7CF
:0A1B1600D9CFE6FFE1CFD9FF93809D
:101B20009392949A8A908A928B9AFD0EDBCF9BF0C7
:101B3000FE0EDBCF9CF09BC0E9FF9CC0EAFF050EC8
:101B4000E926000EEA22EF6A9BC0E9FF9CC0EAFF8B
:101B5000060EE926000EEA22EF6A9BC0E9FF9CC050
:101B6000EAFF070EE926000EEA220A0EEF6E9BC07E
:101B7000E9FF9CC0EAFF030EE926000EEA22000EF0
:101B8000EE6E010EED6E9BC0E9FF9CC0EAFF030EF6
:101B9000E926000EEA22EECF9DF0EDCF9EF0E55251
:101BA000E7CFD9FF1200D9CFE6FFE1CFD9FFFE0E74
:101BB000DB507E0823E19BC0E9FF9CC0EAFF050ED5
:101BC000E926000EEA22EF6A9BC0E9FF9CC0EAFF0B
:101BD000060EE926000EEA22EF6A9BC0E9FF9CC0D0
:101BE000EAFF7E0EEF6E9BC0E9FF9CC0EAFF070E86
:101BF000E926000EEA220B0EEF6EA4D09BC0E9FF8F
:101C00009CC0EAFF070EEB500F0A01E181D0010AE8
:101C10002EE0020A1AE0070A02E0010A93D09BC0F4
:101C2000E9FF9CC0EAFFEE52010EE926000EEA220F
:101C3000FE0EDBCFEFFF9BC0E9FF9CC0EAFF070E63
:101C4000E926000EEA220C0E7CD09BC0E9FF9CC066
:101C5000EAFFEE52FE0EDBCFEFFF9BC0E9FF9CC018
:101C6000EAFF070EE926000EEA220E0E6AD09BC09C
:101C7000E9FF9CC0EAFF050EEB50106EEE52EECF6E
:101C800011F0EFCF12F01150105C000E125423E24D
:101C90009BC0E9FF9CC0EAFF050EEB500001EA6A19
:101CA0009D25E96E9E51EA22FE0EDBCFEFFF9BC021
:101CB000E9FF9CC0EAFF060EE926000EEA22FE0EAE
:101CC000DB50EF269BC0E9FF9CC0EAFF050EE9262A
:101CD000000EEA22EF2A9BC0E9FF9CC0EAFF050E36
:101CE000EB50106E116AEE52EECF12F0EFCF13F000
:101CF0001250101827E11350111824E19BC0E9FF7E
:101D00009CC0EAFF070EE926000EEA220F0E19D04A
:101D10009BC0E9FF9CC0EAFF060EE926000EEA22FE
:101D2000EF28E86C106EFE0EDB50105C01E10ED85F
:101D30009BC0E9FF9CC0EAFF070EE926000EEA22DD
:101D40000A0EEF6EE552E7CFD9FF1200D9CFE6FFBA
:101D5000E1CFD9FFE6529DC0E9FF9EC0EAFFEF50F8
:101D60008A0A40E01F0A38E0340A30E0360A28E0E8
:101D7000060A20E0030A18E0190A10E01B0A08E02E
:101D8000180A47E19DC0E6FF9EC0E6FF3C0E2FD03B
:101D90009DC0E6FF9EC0E6FF3D0E29D09DC0E6FF38
:101DA0009EC0E6FF3E0E23D09DC0E6FF9EC0E6FF2C
:101DB0003F0E1DD09DC0E6FF9EC0E6FF400E17D02F
:101DC0009DC0E6FF9EC0E6FF410E11D09DC0E6FF1C
:101DD0009EC0E6FF420E0BD09DC0E6FF9EC0E6FF10
:101DE000430E05D09DC0E6FF9EC0E6FF440EE66EA2
:101DF0009BC0E9FF9CC0EAFFEE52EF50E66E80EC1C
:101E000009F0E552E552E552E552DF6EDFCF10F002
:101E10001034E552E552E7CFD9FF1200D9CFE6FFE3
:101E2000E1CFD9FF020EE126010EDB6A7E0EE66EDF
:101E300089EC18F0E552A850020BFDE06BD80009C0
:101E4000FAE1E66A89EC18F0E552A850020BFDE0D1
:101E500061D80009FAE1FC0EDBCFE6FF89EC18F04F
:101E6000E552A850020BFDE055D80009FAE1DF6AFF
:101E7000FC0EDB50DF5C2DE2DF50E76EFD0EDBCFAA
:101E8000E9FFFE0EDBCFEAFFE750E926000EEA226B
:101E9000EF50E66E89EC18F0E552DF50E76EFD0E6C
:101EA000DBCFE9FFFE0EDBCFEAFFE750E926000EAD
:101EB000EA22010EDBCFE7FFEF50E726010EE7CF66
:101EC000DBFFA850020BFDE025D80009FAE1DF2A6C
:101ED000CFD7010EDB28E86CE66E89EC18F0E552EE
:101EE000A8A2FED7020EE15C02E2E16AE552E16ED1
:101EF000E552E7CFD9FF1200D9CFE6FFE1CFD9FFF6
:101F0000FE0EDB5002E08A8201D08A92E552E7CFD2
:101F1000D9FF1200D9CFE6FFE1CFD9FFE6528150B9
:101F2000010BDF6EDF5002E0010E01D0000EE55222
:101F3000E552E7CFD9FF12008B8A12008B9A12006C
:101F4000D9CFE6FFE1CFD9FFFD0EDBCFA3F0FE0E28
:101F5000DBCFA4F0A3C0E9FFA4C0EAFFEE6AED6AFC
:101F6000A3C0E9FFA4C0EAFF020EEB6A030EEB6A0E
:101F7000A3C0E9FFA4C0EAFF040EEB6A050EEB6AFA
:101F8000A3C0E9FFA4C0EAFF060EE926000EEA227C
:101F9000000EEE6E0C0EED6EE552E7CFD9FF12008B
:101FA000D9CFE6FFE1CFD9FFA3C0E9FFA4C0EAFF84
:101FB000040EE926000EEA22EECF10F0EFCF11F06A
:101FC000D8801056020E11561050111002E1FF0E6B
:101FD00049D0A3C0E9FFA4C0EAFF040EE926000E21
:101FE000EA22EE2AED22A3C0E9FFA4C0EAFF060E12
:101FF000E926000EEA22EECF10F0EFCF11F0A3C0D9
:10200000E9FFA4C0EAFF020EE926000EEA22105002
:10201000EE24E76E1150EE20EA6EE7CFE9FFFE0EE8
:10202000DBCFEFFFA3C0E9FFA4C0EAFF020EE92661
:10203000000EEA22EE2AEF22A3C0E9FFA4C0EAFFC5
:10204000020EE926000EEA22EE500BE1020EED1818
:1020500008E1A3C0E9FFA4C0EAFF020EEB6A030E89
:10206000EB6A000EE552E7CFD9FF1200D9CFE6FFA9
:10207000E1CFD9FFE652FE0EDBCF10F0A3C0E9FF9F
:10208000A4C0EAFF040EE926000EEA22EECF11F00A
:10209000EFCF12F0D8801156020E12561050115C7C
:1020A000000E125802E2FF0E64D0FE0EDB50106EDE
:1020B000116AA3C0E9FFA4C0EAFF040EE926000EDE
:1020C000EA221050EE261150ED22DF6AFE0EDB50A0
:1020D000DF5C4EE2DF50E76EFC0EDBCFE9FFFD0E6A
:1020E000DBCFEAFFE750E926000EEA22EF50E66E6A
:1020F000A3C0E9FFA4C0EAFF060EE926000EEA220B
:10210000EECF10F0EFCF11F0A3C0E9FFA4C0EAFFBB
:10211000020EE926000EEA221050EE24E76E11505E
:10212000EE20EA6EE7CFE9FFE552E750EF6EA3C07D
:10213000E9FFA4C0EAFF020EE926000EEA22EE2A19
:10214000EF22A3C0E9FFA4C0EAFF020EE926000EB9
:10215000EA22EE500BE1020EED1808E1A3C0E9FF00
:10216000A4C0EAFF020EEB6A030EEB6ADF2AAED7C9
:10217000000EE552E552E7CFD9FF1200D9CFE6FFB6
:10218000E1CFD9FFE652FE0EDBCF10F0A3C0E9FF8E
:10219000A4C0EAFF040EE926000EEA22EECF11F0F9
:1021A000EFCF12F01050115C000E125802E2FF0E39
:1021B00057D0FE0EDB50106E116AA3C0E9FFA4C019
:1021C000EAFF040EE926000EEA221050EE5E1150DE
:1021D000ED5ADF6AFE0EDB50DF5C41E2A3C0E9FF8F
:1021E000A4C0EAFF060EE926000EEA22EECF10F0A8
:1021F000EFCF11F0A3C0E9FFA4C0EAFF1050EE2416
:10220000E76E1150EE20EA6EE7CFE9FFEF50E66E81
:10221000DF50E76EFC0EDBCFE9FFFD0EDBCFEAFF00
:10222000E750E926000EEA22E552E750EF6EA3C020
:10223000E9FFA4C0EAFFEE2A000EEF22A3C0E9FFE7
:10224000A4C0EAFFEE5009E1020EED1806E1A3C0BA
:10225000E9FFA4C0EAFFEE6AED6ADF2ABBD7000EF1
:10226000E552E552E7CFD9FF1200A3C0E9FFA4C0B1
:10227000EAFF040EE926000EEA22EECF10F0EFCFBF
:1022800011F0D8801056020E115610C0F3FF11C085
:04229000F4FF120045
:0C229400A58A9F86F1949F90A292F19081
:1022A000F09C9D86F286F0861200D08EF28EF28C23
:1022B0001200F250800B800A01E0010E106E116ACC
:1022C00010BE116810C0F3FF11C0F4FF1200F250ED
:1022D000400B400A01E0010E106E116A10BE116839
:1022E00010C0F3FF11C0F4FF1200F2BC04D0E1DF14
:1022F000F350F41002E0F36A02D0010EF36EF46AB8
:102300001200F3DFF3CF10F0F4CF11F0F350F4101C
:1023100007E1CFDFF350F41003E1010EF36E01D0BB
:10232000F36AF46A1200DACFE4FFE2CFDAFFE9CF12
:10233000E4FFEACFE4FFF6CFE4FFF7CFE4FFF8CF06
:10234000E4FFF5CFE4FFF3CFE4FFF4CFE4FFFACFEF
:10235000E4FFFBCFE4FF00EE00F0100EE80403E31F
:10236000EECFE4FFFBD700EE10F0040EE80403E329
:10237000EECFE4FFFBD7E652A4AA03D07BEC16F025
:10238000A49A9EA603D0A9EC01F09E96E55200EE19
:1023900013F0040EE80403E3E5CFEDFFFBD700EEF6
:1023A0000FF0100EE80403E3E5CFEDFFFBD7E5CF18
:1023B000FBFFE5CFFAFFE5CFF4FFE5CFF3FFE5CF75
:1023C000F5FFE5CFF8FFE5CFF7FFE5CFF6FFE5CF67
:1023D000EAFFE5CFE9FFE5CFDAFF1100D8CFE4FF50
:1023E000E0CFE4FFE46EDACFE4FFE2CFDAFFE9CF3B
:1023F000E4FFEACFE4FFF6CFE4FFF7CFE4FFF8CF46
:10240000E4FFF5CFE4FFF3CFE4FFF4CFE4FFFACF2E
:10241000E4FFFBCFE4FF00EE00F0100EE80403E35E
:10242000EECFE4FFFBD700EE10F0040EE80403E368
:10243000EECFE4FFFBD7E652F0A003D00EEC14F091
:10244000F090F2A003D035EC14F0F290F2A403D097
:10245000C6EC14F0F2949EA003D0DFEC14F09E9032
:10246000A1A203D002EC15F0A192E55200EE13F008
:10247000040EE80403E3E5CFEDFFFBD700EE0FF019
:10248000100EE80403E3E5CFEDFFFBD7E5CFFBFF3C
:10249000E5CFFAFFE5CFF4FFE5CFF3FFE5CFF5FF9A
:1024A000E5CFF8FFE5CFF7FFE5CFF6FFE5CFEAFF91
:1024B000E5CFE9FFE5CFDAFFE550E5CFE0FFE5CF77
:0424C000D8FF100031
:0C24C40092909292929492968990899244
:1024D0008994899600019F6BA06BE66A0AD8E55241
:1024E000E66A07D8E552120089820000899200004E
:1024F0001200D9CFE6FFE1CFD9FF020EE126899085
:10250000DE6ADD6ADECF10F0DDCF11F0D890115019
:1025100004E6080E105C000E115814E2FE0EDB50AB
:10252000010BE8B08984E8A08994DEDFFE0EDBCFE2
:10253000F3FFF390F342F3CFDBFFDF2A010EE2E378
:10254000DB2AE0D78980020EE15C02E2E16AE55213
:10255000E16EE552E7CFD9FF1200D9CFE6FFE1CF18
:10256000D9FFE652DF6A00019F6BA06B0A0E106E66
:102570000C6EFE0EDBCF07F009EC19F00350DF6E96
:10258000DF50090A34E0010A2DE00F0A26E0010AB3
:1025900022E0030A1EE0010A17E0070A13E0010A1D
:1025A0000CE0030A07E0010A27E1700E00019F1307
:1025B0000D0E21D000019F8D13D0600E00019F13DE
:1025C0000E0E19D0600E14D0500E00019F13030E92
:1025D00012D0300E0DD0300E06D0700E00019F13B9
:1025E000A0810AD0700E00019F130F0E04D0700E50
:1025F00000019F13070EA0130A0E106E0C6EFE0E44
:10260000DBCF07F009EC19F00750DF6EDF50090A45
:102610002EE0010A27E00F0A20E0010A1CE0030A6D
:1026200018E0010A14E0070A10E0010A09E0030AB1
:1026300004E0010A21E10D0E16D000019F8710D0A1
:102640000E0E00019F13C00E16D00E0E11D00B0EF1
:1026500005D0070E0DD0070E06D00D0E00019F13FA
:10266000A08B0AD00F0E00019F13E00E04D00F0EB6
:1026700000019F13600EA01300019F51E66E39DF29
:10268000E552000E00019F15106EFF0EA015116E91
:10269000106E116AE850E66E2CDFE552E552E55205
:1026A000E7CFD9FF120000019F51E66E22DFE5520D
:1026B0000001FF0EA015106E116AE850E66E19DFDA
:0426C000E5521200CD
:0C26C40029D865EF13F0D9CFE6FFE1CF75
:1026D000D9FF020EE126200EDF6EDE52270EDD6EE0
:1026E000D9CFE6FFDACFE6FF020EE66E180EE66EF1
:1026F000C2EC00F0E552E552E552E552F1EC06F08D
:102700000009FCE1020EE15C02E2E16AE552E16EE1
:10271000E552E7CFD9FF1200D9CFE6FFE1CFD9FFCD
:10272000020EE126200EDF6EDE520F0EDD6ED9CFD7
:10273000E6FFDACFE6FF020EE66E690EE66EC2EC49
:1027400000F0E552E552E552E552F1EC06F00009E1
:10275000FCE1020EE15C02E2E16AE552E16EE55263
:10276000E7CFD9FF1200D9CFE6FFE1CFD9FFE6527C
:10277000A80EDF6ED9CFE6FFDACFE6FF010EE66ED8
:10278000180EE66EC2EC00F0E552E552E552E55255
:10279000F1EC06F00009FCE1060EE66E180EE66E9E
:1027A00044EC01F0E552E552F1EC06F00009FCE1E1
:1027B000E552E552E7CFD9FF1200D9CFE6FFE1CFCE
:1027C000D9FFE652A80EDF6ED9CFE6FFDACFE6FFDB
:1027D000010EE66E690EE66EC2EC00F0E552E552BF
:1027E000E552E552F1EC06F00009FCE1060EE66E5A
:1027F000690EE66E44EC01F0E552E552F1EC06F0AC
:0E2800000009FCE1E552E552E7CFD9FF1200D6
:02280E00928AAC
:1028100094940E01020EE76FF19A120053EC16F039
:10282000010EE66E17EC19F0E55260EC16F0000EA2
:10283000E66EE66A500EE66EE66A3BEC09F0E5529B
:10284000E552E552E552120003010F0EFF6FF19EB3
:102850009388938A938C938E8188818A818C818ED0
:102860008A888A8A8A8C8A8E1200D9CFE6FFE1CFC5
:10287000D9FFE652F00E8114E8380F0BDF6EDF50FF
:102880000301FF19010B13E0FFA105D0000EE66E56
:10289000E66A460E04D0000EE66EE66A470EE66E65
:1028A000E66A3BEC09F0E552E552E552E552DF50AD
:1028B0000301FF19020B13E0FFA305D0000EE66E23
:1028C000E66A480E04D0000EE66EE66A490EE66E31
:1028D000E66A3BEC09F0E552E552E552E552DF507D
:1028E0000301FF19040B13E0FFA505D0000EE66EEF
:1028F000E66A4A0E04D0000EE66EE66A4B0EE66EFD
:10290000E66A3BEC09F0E552E552E552E552DF504C
:102910000301FF19080B13E0FFA705D0000EE66EB8
:10292000E66A4C0E04D0000EE66EE66A4D0EE66EC8
:10293000E66A3BEC09F0E552E552E552E552DFCF9D
:0C294000FFF3E552E552E7CFD9FF12008B
:04294C00970EE66E8E
:102950003BEC18F0E552D59E7B0EE66E9B0EE66EC4
:10296000A5EC17F0E552E552CD900201FF6B050E84
:10297000E66E57EC18F0E5527F0EE66E830EE66EBB
:1029800022EC17F0E552E5527990120016D8000EAD
:10299000E66EE66A0A0EE66EE66A3BEC09F0E55280
:1029A000E552E552E5521200000EE66EE66A1FECB3
:1029B00018F0E552E552D58E1200D59E12000201A4
:1029C000FF2B030E106E0C6EFFC207F009EC19F01E
:1029D00003500CE1000EE66EE66A0B0EE66EE66A48
:1029E0003BEC09F0E552E552E552E5521200000ECB
:1029F000E66EE66A03EC18F0E552E552CD8012006F
:102A0000CD9012000401FF5106E138EC16F00401EC
:102A1000010EFF6F04D051EC16F00401FF6BE66A63
:102A2000EA0EE66EE7EC17F0E552E5521200798007
:102A300038EC16F00401010EFF6F1200799051EC92
:082A400016F00401FF6B120007
:082A48001E0EF66E000EF76E83
:102A5000000EF86E00010900F550966F0900F55060
:102A6000976F03E1966701D03DD00900F550916F53
:102A70000900F550926F0900F550936F09000900A5
:102A8000F550E96E0900F550EA6E090009000900E9
:102A9000F550946F0900F550956F09000900F6CFC5
:102AA00098F0F7CF99F0F8CF9AF091C0F6FF92C066
:102AB000F7FF93C0F8FF0001945302E1955307E03C
:102AC0000900F550EE6E9407F8E29507F9D798C023
:102AD000F6FF99C0F7FF9AC0F8FF00019607000EB5
:062AE000975BBFD7120056
:0A2AE600D9CFE6FFDACFE6FFE1CF1B
:102AF000D9FFE2CFDAFFC26AC16AFC0EDB50400D9B
:102B0000F350C00B106EFC0EDB407F0B3C0B101023
:102B1000C26EFD0EDB50040DF350380B116EFD0E2E
:102B2000DB380F0B070B106EFD0EDB50800B101007
:102B30001110C16EFA0EDBCF10F0FB0EDBCF11F0DF
:102B400011C010F0116A10C048FFFA0EDBCF49FF28
:102B5000FC0EDBAE03D09E9C9D8CF28CC280E552B5
:0A2B6000E5CFDAFFE7CFD9FF12003E
:062B6A00D9CFE6FFDACF2F
:102B7000E6FFE1CFD9FFE2CFDAFFA86A9C6AFD0E3B
:102B8000DBB0A888DBA202D0A88C9C8CDBB4A88E1A
:102B9000DBA602D09C8801D09C8ADBA802D0A88446
:102BA00001D0A894DBBA9C86DBAC02D0A38A01D00A
:102BB000A39ADBAE02D0A38801D0A398FB0EDB5012
:102BC000AB6EFC0EDBCF11F011C010F0116A10508B
:102BD0007D6EA88A9C8EE552E5CFDAFFE7CFD9FF5C
:022BE0001200E1
:0E2BE200D9CFE6FFDACFE6FFE1CFD9FFE2CF91
:102BF000DAFFAD6AAC6AFD0EDBB0AD88DBA202D0B5
:102C0000AD8CAC8CDBB4AD8EDBA602D0AC8801D031
:102C1000AC8ADBB8AD84DBBAAC86DBAC02D09D8A73
:102C200001D09D9ADBAE02D09D8801D09D98FB0E0D
:102C3000DB50B06EFC0EDBCF11F011C010F0116A4A
:102C400010507F6EAD8AAC8EE552E5CFDAFFE7CF4C
:042C5000D9FF120096
:0C2C54009490949294948B908B928B94AB
:102C60000E010E0ED16F0F0ED26F120ED36F120027
:102C70003D0EE66EB5EC18F0E552800EE66EE66AA3
:102C8000C6EC16F0E552E5529EA2FED7FC0EE66EAB
:102C90003F0EE66E4EEC17F0E552E552BF80BF8264
:102CA00012002BEF19F0E668A0EC18F0E552800E48
:102CB000E66EE66A97EC16F0E552E552B98012002E
:042CC0000AEF00F027
:0C2CC400400EE66EE66A3C0EE66EF1EC97
:102CD00015F0E552E552E5520E01050EF66FCC6F88
:102CE000400EE66EE66A7C0EE66EB5EC15F0E55237
:102CF000E552E5521200A4AA06D0C8EC17F0E66E21
:102D0000D3EC0DF0E5520101FFA710D0AC98AC88D0
:102D10009C989C88000EE66EE66A1E0EE66EE66AD9
:0E2D200080EC09F0E552E552E552E552120052
:022D2E00D9CFFB
:102D3000E6FFDACFE6FFE1CFD9FFE2CFDAFFE652D6
:102D4000E652FC0EDBCF10F0FD0EDBCF11F0060ECD
:102D5000D89010361136E804FBE110C0DEFF11C038
:102D6000DDFF010EDB50B56EDF50E840E8403F0B61
:102D7000300B106ECF0EB4141010B46EE552E55245
:0C2D8000E552E5CFDAFFE7CFD9FF1200E3
:042D8C00D9CFE6FFB6
:102D9000DACFE6FFE1CFD9FFE2CFDAFFE652E65223
:102DA000FC0EDBCF10F0FD0EDBCF11F0060ED8903D
:102DB00010361136E804FBE110C0DEFF11C0DDFF64
:102DC000010EDB50BB6EDF50E840E8403F0B300B9C
:102DD000106ECF0EBA141010BA6EE552E552E552DD
:0A2DE000E5CFDAFFE7CFD9FF1200BC
:062DEA009280FE0EE66E71
:102DF0001F0EE66E840EE66EE10EE66E73EC15F0C5
:102E0000E552E552E552E55212002DEF19F007EFB9
:102E100000F0D9CFE6FFE1CFD9FF030EE12622EC87
:102E200019F0F3CFDEFFF4CFDDFF020EF36EDB6EA1
:102E3000030EE15C02E2E16AE552E16EE552E7CFA2
:042E4000D9FF1200A4
:0C2E4400D9CFE6FFDACFE6FFE1CFD9FFDF
:102E5000E2CFDAFFFC0EDB50F30B976EFD0EDB507A
:102E60007F0BE824796EFD0EDBB4CD867B6A7A6A2F
:102E7000A192A492DBAE02D0A08201D0A092FC0E5F
:102E8000DBA402D0A38201D0A39297BE978679805B
:0C2E9000E552E5CFDAFFE7CFD9FF1200D2
:042E9C00D9CFE6FFA5
:102EA000DACFE6FFE1CFD9FFE2CFDAFFFD0EDB801C
:102EB000DB82DB84DB86DB88DB8AFC0EDB84DB8663
:102EC000DB88DB8ADB8CDB8EFD0EDBCFE6FFC00E02
:102ED000BA10E552E714BA6EFC0EDBCFE6FF0F0E18
:102EE000BA10E552E714BA6EE552E5CFDAFFE7CF44
:042EF000D9FF1200F4
:0C2EF400D9CFE6FFDACFE6FFFA0EE3CFFD
:102F0000D9FFFB0EE3CFDAFFFC0EE3CFE9FFFD0EA6
:102F1000E3CFEAFFE9CFF3FFEACFF4FFF80EE35087
:102F200003E1F90EE35008E0F80EE30602E2F90EC1
:102F3000E306DECFEEFFF2D7FF0EE3CFDAFFE55276
:0A2F4000FF0EE3CFD9FFE5521200A7
:062F4A00D9CFE6FFDACF4B
:102F5000E6FFE1CFD9FFE2CFDAFFFC0EDB50F30B47
:102F60009A6EFD0EDB507F0BE824CD6ECF6ACE6AE1
:102F70009E90FD0EDBAE02D09D8001D09D909ABE4A
:102F80009A86CD80E552E5CFDAFFE7CFD9FF120070
:102F9000D9CFE6FFDACFE6FFE1CFD9FFE2CFDAFF04
:102FA000E652F20E0101FF179CAC03D0FF919CB0DA
:102FB000FF819CB4FF859CB2FF87AA50DF6EDF5073
:0E2FC000E552E552E5CFDAFFE7CFD9FF120068
:022FCE00D9CF59
:102FD000E6FFDACFE6FFE1CFD9FFE2CFDAFFE65234
:102FE000E652FC0EDBCFDEFFDBCFDDFF010EDB5058
:102FF0007B6EDF507A6EE552E552E552E5CFDAFF9F
:06300000E7CFD9FF12002A
:0A300600D9CFE6FFDACFE6FFE1CFF5
:10301000D9FFE2CFDAFFE652E652FC0EDBCFDEFF4D
:10302000DBCFDDFF010EDB50CF6EDF50CE6EE55201
:0E303000E552E552E5CFDAFFE7CFD9FF1200F7
:02303E00D9CFE8
:10304000E6FFDACFE6FFE1CFD9FFE2CFDAFFE652C3
:10305000E652FC0EDBCFDEFFDBCFDDFF010EDB50E7
:10306000D76EDF50D66EE552E552E552E5CFDAFF76
:06307000E7CFD9FF1200BA
:0A307600D9CFE6FFDACFE6FFE1CF85
:10308000D9FFE2CFDAFFFD0EDB507F0BD56ED76A9A
:10309000D66AF294FD0EDBAE02D0F28A01D0F29A2B
:0E30A000D58EE552E5CFDAFFE7CFD9FF12005B
:0230AE00D9CF78
:1030B000E6FFDACFE6FFE1CFD9FFE2CFDAFFFD0E80
:1030C000DB50FB0BCA6ECC6A9E92FD0EDBAE02D0CB
:1030D0009D8201D09D92CA84E552E5CFDAFFE7CF09
:0430E000D9FF120002
:0C30E400FF0EE350156EEF0E01D0F30E4E
:1030F000E76EE72E79EF18F00C0E146EE76AE72EF4
:103100007FEF18F0142E7EEF18F0152E77EF18F0E1
:023110001200AB
:0E311200D9CFE6FFDACFE6FFE1CFD9FFE2CF5B
:10312000DAFFA8AC04D0A8900101FFB3A880FD0E7F
:10313000DB50A96EE552E5CFDAFFE7CFD9FF1200E9
:10314000D9CFE6FFDACFE6FFE1CFD9FFE2CFDAFF52
:103150000C0EB46ECA94FD0EDB50CB6ECA84E552E1
:0A316000E5CFDAFFE7CFD9FF120038
:06316A00D9CFE6FFDACF29
:10317000E6FFE1CFD9FFE2CFDAFF0C0EBA12CA9414
:10318000FD0EDB50CB6ECA84E552E5CFDAFFE7CF08
:04319000D9FF120051
:0C3194009CEC0FF0E66A79EC12F0E552BA
:1031A000E66A79EC12F0E5521200DDEC14F09EECC8
:0631B0000FF053EF13F0D5
:0A31B600FF0EE350156E480E01D025
:1031C0004C0EE76EE72EFED7E76AE72EFED7152EE8
:0631D000F7D70000120019
:0A31D600C00EF36E00EE00F00E0EC6
:1031E00001D81200EA6002D0EE6AFCD7F350E96021
:0631F0001200EE6AFCD79C
:0A31F6001EEE00F02EEE00F0F86A65
:103200000F9C24EC15F003EC00F0A5EC0AF0FBD7C2
:023210001200AA
:0E321200036A080EE76ED890073603360C509C
:0E322000035C02E3036E072AE72EF7D71200C5
:02322E00FF0E91
:10323000E350E84E1200000000D000D000D0E82E8D
:04324000FAD71200A7
:0C324400C450136E126AC3501210F36ED7
:0632500013C0F4FF1200A0
:04325600BA6A12003E
:04325A00C28212001A
:01325E00006F
:01325F00006E
:01326000006D
:01326100006C
:01FFF800A068
:01FFFA00DD29
:01FFFD00F80B
:00000001FF
